:020000040000FA
:020000000428D2
:08000800FF3083120313A20074
:10001000FF30A3002210C72183120313A210C621B0
:10002000831203132211C52183120313A211C421C9
:1000300083120313A213C321831203132310C221BB
:1000400083120313A310C121831203132311C021B0
:1000500083120313A311BF21831203132312BE21A2
:1000600083120313A312BD21831203132313BC2194
:1000700083120313A313BB21013083120313A600C1
:100080000A30A7002830A800A014A901AA01053051
:10009000AB00512083120313A60A2521DF204A2832
:1000A00050280A3083120313AC000230831203136A
:1000B000AD00831203132414A421831203132C080C
:1000C0005F21831203132410A42183120313A414A9
:1000D000A321831203132C085F2183120313A4109E
:1000E000A321831203132415A221831203132C08C6
:1000F0005F21831203132411A22183120313A41579
:10010000A121831203132C085F2183120313A4116E
:10011000A1218312031325149F21831203132C089A
:100120005F218312031325109F2183120313A5144B
:100130009E21831203132C085F2183120313A51041
:100140009E218312031325159D21831203132C086E
:100150005F218312031325119D2183120313A5151B
:100160009C21831203132C085F2183120313A51112
:100170009C218312031325169B21831203132C0841
:100180005F2183120313061BC92883120313861FE2
:10019000CA28DE288312031325129B21831203131E
:1001A000A5169A21831203132C085F2183120313CF
:1001B000A5129A2183120313AD0B592808000621BA
:1001C0000A3083120313AC0023305F218312031320
:1001D000061FF2281E2183120313A417A021053045
:1001E0005F21002983120313861FFE281721831223
:1001F0000313A417A02105305F21002905305F21DA
:1002000083120313AC0BE42808305F298312031315
:1002100026080139003C031D122983120313A41779
:10022000A021162983120313A413A021080083120E
:100230000313A60183120313A70A252983120313AC
:10024000A60183120313A80A25298312031323137B
:10025000BC2183120313A313BB21831203132608AB
:100260003C3C031D392983120313A6018312031397
:10027000A80A8312031328083C3C031D4529831256
:100280000313A80183120313A70A83120313270879
:100290000D3C031D4F29013083120313A700831265
:1002A00003132708A921831203132808A521831209
:1002B00003132317BC2183120313A317BB29831233
:1002C0000313AE00831203132E0883120313AF002F
:1002D00083120313AF08031D6E29742901307521A1
:1002E00083120313AF036829080083120313B000BD
:1002F00083120313300883120313B1000A308312F0
:100300000313B2000130842983120313B300FF30BA
:1003100083120313B4003208B6003108B5003B3035
:10032000340703189029B50B8F29B60B8D29B30B11
:100330008B290800AD29AD29AD29AD29AD29AD29FD
:10034000B429B429B429B429B42983120313A5000C
:10035000AD2983120313A400B429831203132508C3
:1003600083120313860008008312031324088312E8
:10037000031385000800C829C829C829C829C82925
:10038000C829C829C829CD29CD29CD29CD29CD29CC
:100390008312031323086600080083120313220844
:0403A00065000800EC
:02400E00103F61
:00000001FF
